:020000000A28CC
:0C001400003066001F30650086010E30D1
:10002000920080309300FF309700051C00001928D3
:100030000E28970B15285C200C088D000F089000E7
:10004000FF309700051C000026280E28970B222859
:100050005C200C088E000F0891000D080E02031999
:1000600032280E2810081102031937280E28050817
:1000700094009409940D940D783094051308940419
:100080000E089500F8309505140815020319492843
:100090000E281208110203194E280E280E0894008B
:1000A00007309405940A95010314950D0310940BE1
:1000B00055281508860020288C018F010C309600E9
:1000C000051863286028051C6628632850309400B2
:1000D000940B682805089400140C8F0C8C0C363097
:1000E0009400940B7128960B63280430940003103D
:1000F0008F0C8C0C940B7728C8309400940B7E28BE
:020100000800F5
:02400E000100AF
:00000001FF
